:1000000075C09BC091C299C098C09CC096C095C055
:1000100094C093C092C091C038C18FC08EC0000000
:1000200000000000000000000000000023456C9864
:10003000C9FF040714233764A0FFFFFFFFFFFFFF82
:10004000FFFFFFFFFF000000000000000000234052
:100050005F7AB4FFFFFFFFFFFF00140008140008E1
:100060000E140004080E14000305080E1400040802
:100070000A0E1114000305080A0E101400030508E7
:100080000A0E1012140008000E00080E0004080EDC
:10009000000305080E0004080E1100080E1100F3FD
:1000A000F404080E10121400080A0C0E0F1012149B
:1000B00000080EED14000203040500041400040EF1
:1000C0001400040810140004080F1114000305089C
:1000D0000A0E0004080A0E00EEEDECEB140E080404
:1000E0000004080E00EBECEDEEF3F41411241FBE37
:1000F000CFE5D2E0DEBFCDBF20E0A0E6B0E001C09A
:100100001D92A937B207E1F7EAE7F0E085E58087BD
:1001100081E0838314821282868311828BE081873F
:1001200088E58287E0E6F0E08DEF87838EEF8583B8
:10013000712C55245A94AAD01FC262CF1BBC19BC83
:1001400018BC0895189525B7277E25BF29B72260CA
:1001500029BF21E022BF019728F020E18895215096
:10016000E9F7F9CF089588EE93E0EDCF369A369906
:10017000FECF85B10895CF93C72D81E0870D8F7392
:10018000782E662D90E0EAD16FEF8C2F90E0CF9122
:10019000E5C1FF920F931F93CF93DF93F82E0BE7E8
:1001A00010E0CEE7D0E0F11005C0CE01CFD1F801CC
:1001B000808304C0F8016081CE01D0D121970F5F08
:1001C0001F4FC437D10579F7DF91CF911F910F9160
:1001D000FF900895D0DF81E0DCCF811101C0AECF68
:1001E000815090E0FC01E25EFF4FE491EBBDFC0129
:1001F000EE5CFF4FE491E9BDFC01EA5BFF4F8491A7
:1002000088BD08950F931F93CF93C82F8B01CC23E4
:1002100059F085E0E2DFC80196DF90DFC80193DF87
:10022000C80191DFC150F3CFCF911F910F91089575
:10023000CF93DF93D82F64E170E08AE0E3DF84EFAF
:1002400091E081DF8D2F64E675D1CAE06C2F72D109
:10025000892F68EC70E0D6DF86DF8D2F6C2F6AD196
:10026000D92F68D1892F68EC70E0CCDF7CDF68EC97
:1002700070E08D2FC7DF77DF64E170E08AE0C2DFD6
:1002800084EF91E0DF91CF915ECF189510927900C5
:100290008FEF581204C0612C6EDF81E1582E87E782
:1002A00090E054D1853519F0612C94DF11C0712C88
:1002B000872D90E04BD1682E8F3F19F080E069DFE9
:1002C00007C0872D91E0970D792E803488F3F6CF03
:1002D00090918300D0917D0010917E00C0917B00B1
:1002E000CC2319F010E0D0E09AE19F5F80E040E07D
:1002F00050E06AE570E0992379F09B012F5F3F4F52
:10030000F9013197E491EE2319F0822F861BF6CF85
:100310009150AB01B901EFCF982F6D2F70E0A82F4E
:10032000B0E0E92FF0E0112321F09D012E1B3F0BDF
:1003300005C09F0121503109260F371F3197E40F67
:10034000F51F049127593F4FF9010083915049F758
:100350008D0F80938500DD2371F0112329F0282F64
:1003600030E02150310902C020E030E0F901E759C6
:10037000FF4F91E0908397E0980F292F2150E22FB3
:10038000E81BF0E0EB51FF4FE491A22FB0E0A7593A
:10039000BF4FEC932813F2CFE92FF0E0E859FF4F5D
:1003A00021E0409169003081431320E0921B90933B
:1003B0008600262D253FE8F5352D3131B0F490919A
:1003C00087009F3F29F4809179008093870006C0C1
:1003D00091E0960D692E981708F0612C80918700A6
:1003E0008F5F8F718093870024C0209179002093C4
:1003F00087003133C0F420918000222311F0CC23F8
:1004000039F091E0960D692E981798F0612C11C083
:10041000262D6816D9F3662019F02150622E09C0E6
:100420009150692E06C0C111F1CF80917C008823C4
:1004300069F3512C8FEF8DBD80E68CBDAB9A8FE3B5
:1004400084BB8BE187BB88EE88BB81E083BF91EAE8
:100450009ABD80BF8BB780628BBF8AB785608ABF29
:1004600085B7806285BF789497B986EC86B98CE2AF
:1004700091E069DE7BDEDCDEFACF112416B85EDEA9
:1004800087B38C7E87BB80E051E041E020E030E024
:10049000A8E0999B06C0F9013197F1F79AB79560EA
:1004A0009ABF96B39A27999B03C0511003C034C0DA
:1004B000911107C040E3451588F581112FC050E028
:1004C00049E0652D71E0623308F070E0760F572E39
:1004D000511108C0811105C081E0911103C080E075
:1004E00001C081E0999895B7977E906195BFA895D6
:1004F000942F987011F490E401C090E6916091BD42
:1005000095B7946895BF9B7F95BF78948895F8942C
:1005100091B59F7B91BDBDCF9111D3CF8FE58DBF9D
:1005200082E08EBF1FBEB2DE999A552011F0189559
:1005300001C0A3DF991B79E004C0991F961708F04A
:10054000961B881F7A95C9F780950895E199FECF8B
:100550009FBB8EBBE09A99278DB30895262FE19912
:10056000FECF1CBA9FBB8EBB2DBB0FB6F894E29A90
:0C057000E19A0FBE01960895F894FFCFA9
:00000001FF
